:020000020000FC
:1000000012C018951895189518951AC01895189536
:06001000189518951895E3
:1000180018951895189518951895189518950FED21
:100028000DBF00E809BFF89400E00DBD00E00CBD6D
:1000380003E00EBD7894FFCF25D17EE9E1D060E0E2
:10004800FDD07FE9D8D08894F9D0262F0894F6D02F
:10005800362F10D136953695369536953695122F1A
:10006800110F110F110F130F26952695269526951A
:100078002695022F2227332740E0310F201F439572
:100088004D37D9F744273051274212F04395FBCF1B
:10009800305F284D409360004427385E234012F0BB
:1000A8004395FBCF38512C4F409361004427345679
:1000B800204012F04395FBCF3C592F4F40936200EC
:1000C80044273A50204012F04395FBCF40936300F9
:1000D8000FEF01BB01D0189581D07BD07AD048E0D2
:1000E80000916300112766271395600F1830E1F718
:1000F80011274A95E4E8F3E0E40FF11FE60FF11F3A
:10010800C89500E000116AD001E0001162D04030CB
:1001180081F749E000916200112766271395600F67
:100128001930E1F711274A95EAE2F3E0E40FF11FED
:10013800E60FF11FC89500E0001150D001E0001152
:1001480048D0403081F748E00091610011276627C8
:100158001395600F1830E1F711274A95EAEDF2E0A0
:10016800E40FF11FE60FF11FC89500E0001136D02B
:1001780001E000112ED0403081F72BD047E00091EC
:100188006000112766271395600F1730E1F71127D4
:100198004A95E4E9F2E0E40FF11FE60FF11FC89574
:1001A80000E000111BD001E0001113D0403081F7AE
:1001B80010D014D013D012D011D04427439509D0B1
:1001C8004830E1F704E002BB06E002BB01E002BBF5
:1001D800089501E002BB05E002BB089503E002BBFD
:1001E80007E002BB089552E05A95F1F7089551E0EF
:1001F8005A95F1F708958C9A8D98F5DF8C98F7DF6A
:10020800672F8D9AF4DF0894661F01C0660F59F0B6
:100218008C9A18F400008D9802C08D9A00C0E3DF14
:100228008C98E1DFF3CF8C9A8D98DDDF8C98849BD6
:10023800FECF889485990894D6DF089570FFE3CFA0
:10024800881F61E08C9A000000008D98CCDF8C98A4
:10025800CADF889485990894661FA0F78C9A8795B9
:1002680010F48D9801C08D9ABEDF8C98849BFECFC8
:10027800BADF08958C9A8D9AB6DF8C98B8DF8D987E
:10028800B2DF0895882782BB81BB08950000000073
:10029800000000000000000001010101010001014F
:1002A800000100010001010100000101000101013C
:1002B800000101010001010101010100010000002C
:1002C8000001010101010101010101000001010119
:1002D800010101010001000101010000000000000E
:1002E80001010101010000010100010001000001FC
:1002F80001010000010100000101010001010001EC
:1003080000010101010100010001000000000001DD
:1003180001010101010100010101000001010001C9
:1003280001010100010001010100010000000000BD
:1003380000010001010001010001010000010000AD
:10034800010001010001000000010100010001019C
:10035800000001010100000101000101010100008C
:10036800010000000000010100010100010101017C
:10037800010001000000010101010001010100016B
:10038800010101010000000001000101010101005B
:10039800010101000100010001010101000001014A
:1003A8000100010101000101010100010101010138
:1003B800010100010000000001010101010101012A
:0C03C8000101010100000101010101011F
:00000001FF
